:020000040800F2
:1000000060450020D519000881030008830300081B
:10001000870300088B0300088F030008000000001E
:100020000000000000000000000000009303000832
:1000300095030008000000009703000899030008DA
:10004000EF190008EF190008EF190008EF19000870
:10005000EF190008EF190008EF190008EF19000860
:10006000EF190008EF190008EF190008EF19000850
:10007000EF190008EF190008EF190008EF19000840
:10008000EF190008EF190008EF190008EF19000830
:10009000EF190008EF190008EF190008EF19000820
:1000A000EF190008EF190008EF190008EF19000810
:1000B000010A0008EF190008EF190008EF190008FD
:1000C000EF190008EF190008EF190008EF190008F0
:1000D000EF1900085D060008EF190008EF19000885
:1000E000EF190008EF190008EF190008EF190008D0
:1000F000EF190008EF190008EF190008EF190008C0
:10010000EF190008EF190008EF190008EF190008AF
:10011000EF190008EF190008EF190008EF1900089F
:10012000EF190008EF190008EF190008EF1900088F
:10013000EF190008EF190008EF190008EF1900087F
:10014000EF190008EF190008EF190008EF1900086F
:10015000EF190008EF190008EF190008EF1900085F
:10016000EF190008EF190008EF190008EF1900084F
:10017000EF190008EF190008EF190008EF1900083F
:10018000EF190008EF19000800F002F800F042F83B
:100190000AA090E8000C82448344AAF10107DA45E2
:1001A00001D100F037F8AFF2090EBAE80F0013F0F2
:1001B000010F18BFFB1A43F001031847483D000028
:1001C000683D0000103A24BF78C878C1FAD85207B9
:1001D00024BF30C830C144BF04680C6070470000C1
:1001E0000023002400250026103A28BF78C1FBD840
:1001F000520728BF30C148BF0B6070471FB503F0DE
:100200007BFE9DE8030003F067FD03F0D0FC1FBDFB
:1002100010B510BD03F0EEFD1146FFF7EFFF00F043
:1002200023F803F00CFE03B4FFF7F2FF03BC03F066
:100230003DFE00000B49D1F800C04A685CF8043B61
:100240001068184442F8040B8C4528BFA1F1DC0C5F
:100250008A4228BFA1F1DC02C1F800C04A6020F048
:1002600000407047F43E002000F099FA00F07AFB5D
:1002700000F094FB4FF4A06001F0CCFB4FF4E130B0
:1002800000F094F936490868804736490868804785
:10029000354803F083FB01F07DFB01F08AFB5EE053
:1002A000002000F092FE50B3132804D0172806D087
:1002B0001C282CD11FE0002001F094F828E0002039
:1002C00000F07AFE00F0010018B10121002000F0DA
:1002D0003FFF002000F0ACFE24490880084600885B
:1002E000002807DD084602882149002001F091F925
:1002F00000F03CFA0CE0002001F00FF908E02023A8
:100300004EF660220121002001F00CF800E000BF51
:1003100000BF4FF4385000F092FC00F0010060B9CB
:10032000002001F0FAF820234EF66022012100207F
:1003300000F0F8FF002001F055F80E480078012881
:100340000BD100200B4908700B4802880B49002094
:1003500001F0F6F800200849088001F034FB9FE71F
:100360002400002030000020182A00200000002077
:10037000740000201A0000201800002074280020BB
:10038000704700BFFEE700BFFEE700BFFEE700BF0B
:10039000FEE7704770477047704700000CB50020BB
:1003A000019000907648006840F4803074490860FD
:1003B00000BF7348006800F4003000900198401CB2
:1003C0000190009818B90198B0F5A04FF1D16C4890
:1003D000006800F4003010B10120009001E000201E
:1003E00000900098012846D165484030006840F0F0
:1003F00080506349403108606248006840F44040E2
:10040000604908605E48083000685D49083108604E
:100410000846006840F4004008600846006840F460
:10042000A05008605848091F0860081F006840F085
:100430008070091F086000BF5148006800F000701C
:100440000028F9D040F20570504908604C48083047
:10045000006820F003004A49083108600846006837
:1004600040F00200086000BF45480830006800F016
:100470000C000828F8D10CBD10B54548006840F4C0
:100480007000434908603E48006840F001003C4964
:10049000086000203A4908310860394800683D4941
:1004A0000840374908603C48091D0860081F00687B
:1004B00020F48020091F0860002031490C310860B9
:1004C000FFF76CFF4FF0006031498039086010BDC4
:1004D00070B500200022022300240221284D083597
:1004E0002D6805F00C0020B1042806D0082834D16E
:1004F00007E02A4D2A4E356033E02A4D284E3560FC
:100500002FE01F4D2D1D2D68C5F380541C4D2D1D52
:100510002D6805F03F0154B1224DB5FBF1F5184EA1
:10052000361D3668C6F3881605FB06F209E01B4D3A
:10053000B5FBF1F5124E361D3668C6F3881605FB7D
:1005400006F20F4D2D1D2D68C5F301456D1C6B0086
:10055000B2FBF3F5124E356003E0104D104E3560DE
:1005600000BF00BF064D08352D68C5F303150E4EBC
:10057000705D0B4D2D68C540094E356070BD0000A3
:10058000003802400070004008544007003C024020
:1005900088ED00E0FFFFF6FE103000240024F40098
:1005A0000400002000127A000800002010B588B076
:1005B00004460121022001F0E1FD0121102001F09B
:1005C00037FE07220621DD4801F0A5FB0722114670
:1005D000DA4801F0A0FBC020069002208DF81C0034
:1005E0008DF81D0000208DF81E0001208DF81F00E1
:1005F00006A9D24801F004FB02940020ADF80C00DB
:10060000ADF80E00ADF81000ADF814000C20ADF8F8
:10061000120002A9CA4802F0FEFF25208DF804004E
:1006200006208DF8050000208DF8060001208DF8C9
:10063000070001A801F0F3F9012240F22551C0485A
:1006400003F027F9012240F22441BD4803F021F9CB
:100650000121BB4803F067F808B010BD10B540F2A7
:100660002551B74803F050F9B8B1B6480088322890
:1006700002DB0020B3490880B14803F083F8C1B21F
:10068000B04802880088401CAE4B1880AE488154A8
:1006900040F22551AA4803F02EF940F22441A8481F
:1006A00003F032F940B1A6480088C4B2A44880885B
:1006B000C4B20120A549087010BD2DE9F0410446DF
:1006C0002746384603F008FA064622463146A04837
:1006D00003F09EF900250CE0715D994803F04EF897
:1006E00000BF8021964803F0F9F80028F9D0681C73
:1006F000C5B2A542F0DB304603F01DFA0220BDE88A
:10070000F08130B5002400210023002207E0481CBE
:10071000C1B290480088814201DB002030BD8E4884
:10072000405CAA28F3D1481CC0B201468A4D285C1F
:10073000801C2C5C022205E08748805C1844C3B210
:10074000501CC2B28448405C801C9042F4DC9C4245
:1007500001D00020E2E78048405CC01C7E4D285C50
:10076000552801D00020D9E70120D7E710B5FFF7C1
:10077000C8FF28B1774802887749754803F02BF9FC
:100780007648007850B1002074490870704803F032
:1007900009F918B96F490878FFF78FFF10BD10B538
:1007A0000020C7E00022C0EBC00303EB43036C4C06
:1007B00004EB43039A700122C0EBC00303EB430335
:1007C00004F81320C0EBC00303EB430304EB430323
:1007D0005A700022C0EBC00303EB430304EB430356
:1007E000DA700023C0EBC00202EB420204EB4202CB
:1007F00093710122C0EBC00303EB430304EB4303FB
:100800001A710123C0EBC00202EB420204EB420268
:1008100053710023C0EBC00202EB420204EB420220
:10082000D3710022C0EBC00303EB430304EB43038B
:100830001A72C0EBC00303EB430304EB43035A7289
:10084000C0EBC00303EB430304EB43039A720122A2
:10085000C0EBC00303EB430304EB4303DA72002253
:10086000C0EBC00303EB430304EB43031A73C0EB79
:10087000C00303EB430304EB43035A7300210BE073
:100880000023C0EBC00202EB4202354C04EB4202F3
:100890000E3253544A1CD1B20C29F1DB0122C0EBB9
:1008A000C00303EB43032E4C04EB43039A76C0EBE7
:1008B000C00303EB430304EB4303DA766422C0EB8B
:1008C000C00303EB430304EB43031A770022C0EB9E
:1008D000C00303EB430304EB43035A77C0EBC003AD
:1008E00003EB430304EB4303DA83C0EBC00303EBE6
:1008F000430304EB43031A84C0EBC00303EB43033D
:1009000004EB43035A84C0EBC00303EB430304EB43
:1009100043039A84C0EBC00303EB430304EB43039C
:10092000DA84C0EBC00303EB430304EB43031A85F3
:10093000421CD0B20828FFF635AF10BD00040240BB
:100940000010014018000020742800201A00002028
:10095000182A00200000002074000020230000203E
:10096000A62800201CB50121102001F007FC04205E
:10097000009001208DF8040000208DF8060003206F
:100980008DF805006946044801F03AF9042102484F
:1009900001F0B2F91CBD0000001002401FB501219A
:1009A000084601F034FC4FF0804001F07BFF00204E
:1009B000ADF80C00ADF80600F920029042F2CF002D
:1009C000ADF8040001A94FF0804002F018F81C2097
:1009D0008DF8000001208DF8030005208DF801003E
:1009E00000208DF80200684601F019F80122114636
:1009F000900702F0A5FC0121880702F089F81FBDCD
:100A000010B50121880702F0B2FC98B101218807D6
:100A100002F0BEFC01200849087008480078401C1C
:100A200006490870084600780A2803D104210448C2
:100A300001F06DF910BD000023000020220000200D
:100A40000010024000B587B00121084601F096FB76
:100A50000121022001F092FB0121080301F0E8FBD3
:100A600005220721514801F056F9052206214F4879
:100A700001F051F9052211464C4801F04CF90522CC
:100A800004214A4801F047F91020059001208DF813
:100A9000180000208DF81A0001208DF81B0003209B
:100AA0008DF8190005A9414801F0AAF810213F4826
:100AB00001F022F9C020059002208DF818000320D3
:100AC0008DF8190000208DF81A0001208DF81B0008
:100AD00005A9364801F094F82020059002208DF8F1
:100AE000180003208DF8190000208DF81A0001204D
:100AF0008DF81B0005A92D4801F082F800212C4833
:100B000001F0D6FD0020ADF800004FF48270ADF882
:100B100002000020ADF80400ADF80600ADF80800B2
:100B20004FF40070ADF80A000020ADF80C00ADF8ED
:100B30000E000720ADF8100069461D4801F0BEFC0C
:100B400001211B4801F0B4FD002007B000BD10B525
:100B5000044600BF0221164801F074FE0028F9D0B7
:100B60002146134801F025FE00BF0121104801F085
:100B700069FE0028F9D00E4801F018FEC0B210BD81
:100B800070B506460D461021084801F0B7F800245C
:100B900004E0285DFFF7DBFF2855641CB442F8DB56
:100BA0001021024801F0A8F8002070BD00000240AA
:100BB000003001400146FB48405C7047F94A11543F
:100BC00070470146F84830F8110070470146F74871
:100BD00030F81100704710B51021F54801F08EF87B
:100BE00010BD10B51021F24801F086F810BD10B507
:100BF0000446F04881682046884710BD70B5044619
:100C00000D461021EA4801F079F8EA488168C4F3FA
:100C100007408847E7488168C4F30720884704F005
:100C2000F802121DD0B2E34A91688847E148816812
:100C3000284688471021DE4801F05EF870BD70B587
:100C4000044600251021DA4801F058F8D948816897
:100C5000C4F307408847D7488168C4F30720884712
:100C600004F0F800D34A91688847D2488168002090
:100C7000884705461021CE4801F03EF8284670BD51
:100C80002DE9F04104460F46154600261021C848BC
:100C900001F034F8C7488168C4F307408847C54865
:100CA0008168C4F30720884704F0F802121DD0B20F
:100CB000C04A9168884700BF05E0B85DBD4A9168A9
:100CC0008847701C86B2AE42F7DB1021B84801F0AD
:100CD00013F82846BDE8F0812DE9F04104460F469F
:100CE000154600261021B24801F008F8B148816885
:100CF000C4F307408847AF488168C4F3072088479A
:100D000004F0F800AB4A9168884700BF06E0A948A4
:100D1000816800208847B855701C86B2AE42F6DB69
:100D20001021A34800F0E8FF2846BDE8F08110B587
:100D3000044621460020FFF761FF10BD10B580205A
:100D4000FFF7F5FF10BD2DE9F04105460E460027DF
:100D5000B84600248DE0295D41F6087202EB44108C
:100D6000FFF74CFF315D41F6086202EB4410FFF7DC
:100D700045FF00208D4921F814008B4921F814000B
:100D8000B7F5804F32DC285D042816D004DC01283A
:100D900007D0022823D10AE0082814D010281ED139
:100DA00017E04FF48060814921F814001DE04FF4F2
:100DB00000607E4921F8140017E04FF480507B4911
:100DC00021F8140011E04FF40050784921F8140084
:100DD0000BE04FF48040754921F8140005E04FF412
:100DE0000060714921F8140000BF00BFB8F5804FC2
:100DF00032DC305D042816D004DC012807D002283C
:100E000023D10AE0082814D010281ED117E04FF48F
:100E10008060654921F814001DE04FF400606249CC
:100E200021F8140017E04FF480505F4921F81400B6
:100E300011E04FF400505C4921F814000BE04FF42E
:100E40008040594921F8140005E04FF400605649EC
:100E500021F8140000BF00BF544830F81400384493
:100E600007B2514830F8140040440FFA80F8601C73
:100E700004B2082CFFF66FAFBDE8F08110B5044650
:100E8000042221469001FFF7FBFE10BD10B5044679
:100E9000042221469001FFF71FFF10BD10B5044644
:100EA000042221464FF4A060FFF7EAFE10BD10B502
:100EB0000446062221464FF41060FFF7E1FE10BD04
:100EC00010B50446042221464FF47060FFF7D8FEA7
:100ED00010BD10B50446042221469001FFF7FCFE28
:100EE00010BD10B50446042221464FF4A060FFF760
:100EF000F3FE10BD10B50446062221464FF41060E3
:100F0000FFF7EAFE10BD10B50446042221464FF457
:100F10007060FFF7E1FE10BD10B54FF4A850FFF769
:100F20008EFE10BD10B50446210A4FF4C850FFF7DD
:100F300065FEE1B24FF4D050FFF760FE10BD10B572
:100F4000044621464FF4D850FFF758FE10BD70B547
:100F50000446FFF7E1FF60EA0400C5B229464FF4FA
:100F6000A850FFF74BFE70BD70B504460D46290A28
:100F700041F2082202EB4410FFF740FEE9B241F2D1
:100F8000083202EB4410FFF739FE70BD70B504461D
:100F90000D4641F2086101EB44102946FFF72EFE91
:100FA00070BD000058000020062A0020F62900200D
:100FB000000002402400002010B504464FF40271E6
:100FC00001EB4410FFF73BFE10BD10B504464FF493
:100FD000427101EB4410FFF732FE10BD70B50446BC
:100FE0000025002600BF42F2080101EB4410FFF784
:100FF00026FE064642F2081101EB4410FFF71FFEE1
:1010000000EB062086B27EB142F2080101EB4410EB
:10101000FFF715FE054642F2081101EB4410FFF7F9
:101020000EFE00EB052085B2B542DCD1284670BD2E
:1010300070B504460025002600BF42F2086101EBAE
:101040004410FFF7FCFD064642F2087101EB441024
:10105000FFF7F5FD00EB062086B27EB142F2086193
:1010600001EB4410FFF7EBFD054642F2087101EB7E
:101070004410FFF7E4FD00EB052085B2B542DCD15A
:10108000284670BD2DE9F04104460F46164600255E
:10109000A84642F2084101EB4410FFF7D0FD054697
:1010A00042F2085101EB4410FFF7C9FD00EB0520A7
:1010B00085B2280200EB441000F110083246394690
:1010C0004046FFF7DDFDA81985B2290A42F2084221
:1010D00002EB4410FFF792FDE9B242F2085202EB34
:1010E0004410FFF78BFDBDE8F0812DE9F041044687
:1010F0000F4616460025A84642F6080101EB4410AB
:10110000FFF79DFD054642F6081101EB4410FFF77D
:1011100096FD00EB052085B2280200EB441000F19B
:101120001808324639464046FFF7D6FDA81985B261
:10113000290A42F6080202EB4410FFF75FFDE9B20C
:1011400042F6081202EB4410FFF758FDBDE8F081AB
:1011500070B504460D464FF4027101EB4410294668
:10116000FFF74CFD70BD002107E0002200E0521C9B
:1011700042F210739A42FADB491C8142F5DB704758
:1011800010B54FF4FA60FFF7EEFF00BF4FF4385090
:10119000FFF755FD00F001000028F7D08020FFF791
:1011A000C6FD6420FFF7DFFF4D48FFF780FE4C4887
:1011B0000A30FFF773FE4A480E30FFF75FFE4848DB
:1011C000801DFFF77DFE47494748FFF7BCFD4FF400
:1011D000FA60FFF7A7FE0820FFF7B1FEC0214FF429
:1011E000B050FFF70BFD01214FF4C050FFF706FD93
:1011F0001F2142F60840FFF701FD002010BD30B569
:10120000ADF2044D39A0006800900020FFF7DDFE2C
:1012100060B3132804D0172809D01C2839D121E045
:101220004EF661226946002000F0FBF831E0002014
:10123000FFF7C2FE00F0010018B101210020FFF706
:1012400087FF0020FFF7F4FE0446002C09DD4FF471
:10125000806101A802F0F9FCA2B201A9002000F00F
:10126000D8F916E0002000F058F912E0FEF7E2FF8E
:1012700042F2107190FBF1F201FB12004CF250317E
:10128000084485B220232A460121002000F04AF8B4
:1012900000BF00BF4FF43850FFF7D1FC00F0010051
:1012A000D0B9002000F039F9FEF7C4FF42F2107106
:1012B00090FBF1F201FB12004CF25031084485B270
:1012C00020232A460121002000F02CF84EF661224E
:1012D0006946002000F0A5F80DF2044D30BD000075
:1012E000340000205000002048000020C0A8000268
:1012F00010B504464FF4847101EB44101021FFF740
:101300007DFC00BF4FF4847101EB4410FFF797FCA4
:101310000028F7D14FF4027101EB4410FF21FFF7D1
:101320006DFC10BD2DE9F04104460D461646984669
:1013300005F00F0001280FD005F00F0002280BD098
:1013400005F00F00032807D005F00F00042803D094
:1013500005F00F00052841D12046FFF7C9FF45EAF7
:101360000801082202EB4410FFF748FC76B1310A6D
:101370004FF4816202EB4410FFF740FCF1B24FF4EE
:10138000A16202EB4410FFF739FC15E0FE4800882B
:10139000401CFD4908800A461288110A4FF48162F8
:1013A00002EB4410FFF72AFCF74A11784FF4A162D0
:1013B00002EB4410FFF722FC4FF4847101EB441060
:1013C0000121FFF71BFC00BF4FF4847101EB4410B7
:1013D000FFF735FC0028F7D1012700E00027384649
:1013E000BDE8F08170B504464FF4427101EB441042
:1013F000FFF725FC132811D14FF4847101EB441041
:101400000221FFF7FBFB00BF4FF4847101EB441096
:10141000FFF715FC0028F7D1012500E0002528463C
:1014200070BD2DE9F04105460C4616462078FF2890
:1014300008D16078FF2805D1A078FF2802D1E07894
:10144000FF2808D0207828B9607818B9A07808B9A2
:10145000E07800B10EB900275CE00127217840F662
:10146000084202EB4510FFF7C9FB617840F60852CD
:1014700002EB4510FFF7C2FBA17840F6086202EBD1
:101480004510FFF7BBFBE17840F6087202EB451010
:10149000FFF7B4FB310A41F2080202EB4510FFF7F7
:1014A000ADFBF1B241F2081202EB4510FFF7A6FBCB
:1014B0004FF4847101EB45100421FFF79FFB00BF3F
:1014C0004FF4847101EB4510FFF7B9FB0028F7D109
:1014D00017E04FF4427101EB4510FFF7B0FB1728FE
:1014E00000D116E02846FFF767FD00F0080040B184
:1014F0004FF4027101EB45100821FFF77FFB002735
:1015000007E04FF4427101EB4510FFF798FB1528F7
:10151000DFD100BF3846BDE8F08110B504464FF476
:10152000847101EB44100821FFF768FB00BF4FF402
:10153000847101EB4410FFF782FB0028F7D110BD46
:101540002DE9F04704468846164600250027A9469F
:101550002046FFF73BFBB04204DA2046FFF736FB9C
:10156000074600E0374600BF2046FFF737FD8146BB
:101570004FF4427101EB4410FFF761FB0546172D54
:1015800003D01C2D01D0002701E0B945ECDB00BFE2
:101590003A4641462046FFF775FD4FF4847101EB52
:1015A00044102021FFF72AFB00BF4FF4847101EBA8
:1015B0004410FFF744FB0028F7D110E04FF44271CC
:1015C00001EB4410FFF73BFB0546172D07D01C2D00
:1015D00005D02046FFF78CFE0020BDE8F0874FF4D1
:1015E000027101EB4410FFF72AFB00F010001028F5
:1015F000E4D14FF4027101EB44101021FFF7FEFA21
:101600004FF4027101EB44101021FFF7F7FA38464E
:10161000E3E72DE9F04104460E4615460027002D6C
:1016200015DD2A4631462046FFF75FFD4FF48471F1
:1016300001EB44104021FFF7E1FA00BF4FF4847141
:1016400001EB4410FFF7FBFA0028F7D12F4638468C
:10165000BDE8F0812DE9F0470446894616461D464F
:10166000089F4FF000082046FFF7B0FAB04204DAB6
:101670002046FFF7ABFA804600E0B046287828B94C
:10168000687818B9A87808B9E87800B117B94FF0A8
:10169000000863E0297840F6084202EB4410FFF7A7
:1016A000ADFA697840F6085202EB4410FFF7A6FA4B
:1016B000A97840F6086202EB4410FFF79FFAE97838
:1016C00040F6087202EB4410FFF798FA390A41F22B
:1016D000080202EB4410FFF791FAF9B241F2081246
:1016E00002EB4410FFF78AFA424649462046FFF7CC
:1016F000C9FC4FF4847101EB44102021FFF77EFAFE
:1017000000BF4FF4847101EB4410FFF798FA0028F2
:10171000F7D112E04FF4027101EB4410FFF78FFA9A
:1017200000F0080048B14FF4027101EB4410182199
:10173000FFF764FA0020BDE8F0874FF4027101EB77
:101740004410FFF77CFA00F010001028E2D14FF4AB
:10175000027101EB44101021FFF750FA4046EAE70E
:101760002DE9FC5F05468A4691461E46DDF830802D
:1017700000270024A346B9F1000F7CDD42F60801E2
:1017800001EB451002E0000060000020FFF757FA6F
:10179000044642F6081101EB4510FFF750FA00EB42
:1017A000042084B2200200EB451000F1180B082140
:1017B00001EB4510FFF743FA00F00700022804D0C0
:1017C000032844D0042879D179E008226946584694
:1017D000FFF782FA04F1080084B29DF8000030702F
:1017E0009DF8010070709DF80200B0709DF8030034
:1017F000F0709DF80400A8F800009DF8050098F826
:10180000001000EB0120A8F800009DF806709DF87C
:10181000070000EB072087B2200200EB451000F123
:10182000180B3A4651465846FFF756FAE01984B26B
:10183000210A42F6080202EB4510FFF7DFF9E1B298
:1018400042F6081202EB4510FFF7D8F968E00622CD
:1018500069465846FFF740FAA01D84B29DF8000083
:1018600030709DF8010070709DF80200B0709DF816
:101870000300F07000E064E09DF804709DF805003E
:1018800000EB072087B2200200EB451000F1180B97
:101890003A4651465846FFF71FFAE01984B2210A2A
:1018A00042F6080202EB4510FFF7A8F9E1B242F652
:1018B000081202EB4510FFF7A1F931E02FE00222F8
:1018C00069465846FFF708FAA01C84B29DF80070DC
:1018D0009DF8010000EB0720801E87B240F2EA501D
:1018E000874201DD00BFFEE7200200EB451000F15A
:1018F000180B3A4651465846FFF7EEF9E01984B204
:10190000210A42F6080202EB4510FFF777F9E1B22F
:1019100042F6081202EB4510FFF770F900E000BF35
:1019200000BF4FF4847101EB45104021FFF766F9C9
:1019300000BF4FF4847101EB4510FFF780F90028D8
:10194000F7D13846BDE8FC9F1CB50121102000F0FE
:1019500015FC01208DF8040000208DF80600012000
:101960008DF8070003208DF805004020009069469F
:10197000174800F045F9202000906946144800F00F
:101980003FF92021124800F0B7F94021104800F03B
:10199000B5F91CBD10B545F2555000F0F5F9002021
:1019A00000F0F5F94FF4966000F0F4F900F0F5F965
:1019B00010BD10B500F0F6F910BD10B52021044897
:1019C00000F09AF910BD10B500F0E7F910BD000065
:1019D000001002400948804709480047FEE7FEE73B
:1019E000FEE7FEE7FEE7FEE7FEE7FEE7FEE7FEE7CF
:1019F00004480549054A064B704700007904000871
:101A000089010008603F00206045002060410020FF
:101A10006041002032490143324A1160704770B57D
:101A2000002100230F22C4781CB32E4C246804F438
:101A3000E064C4F5E064C4F30721C1F10404E3B237
:101A40000A4144789C40E1B28478144021430C0759
:101A5000210E254C05786155047804F01F050124FA
:101A6000AC4005786D11AD0005F1E025C5F80041E9
:101A700009E0047804F01F050124AC401B4D0678F2
:101A8000761145F8264070BD194A0A400243154BAD
:101A90001B1F1A60704739B1124A121D12680243A7
:101AA000104B1B1D1A6006E00E4A121D126882437D
:101AB0000C4B1B1D1A607047042808D14FF0E02121
:101AC000096941F004014FF0E022116107E04FF095
:101AD000E021096921F004014FF0E0221161704713
:101AE0000000FA050CED00E000E400E080E100E019
:101AF00080FFFF1F10B504469848844208D1012199
:101B0000084600F0A6FB0021012000F0A2FB76E0D1
:101B10009348844208D10121022000F09AFB002161
:101B2000022000F096FB6AE08E48844208D1012131
:101B3000042000F08EFB0021042000F08AFB5EE010
:101B40008948844208D10121082000F082FB00214D
:101B5000082000F07EFB52E08448844208D1012135
:101B6000102000F076FB0021102000F072FB46E010
:101B70007F48844208D10121202000F06AFB002127
:101B8000202000F066FB3AE07A48844208D1012127
:101B9000402000F05EFB0021402000F05AFB2EE0C8
:101BA0007548844208D10121802000F052FB0021B9
:101BB000802000F04EFB22E07048844208D10121D1
:101BC000801500F046FB0021A01500F042FB16E056
:101BD0006B48844208D10121401500F03AFB0021F6
:101BE000601500F036FB0AE06648844207D1012107
:101BF000001500F02EFB0021201500F02AFB10BD7F
:101C0000F0B50A4600210023002400BF3DE0012575
:101C100005FA01F3156805EA03049C4234D105680E
:101C20004F000326BE40B543056015794E00B54010
:101C30000668354305601579012D02D01579022D0E
:101C400016D185684F000326BE40B543856055799F
:101C50004E00B540866835438560456801268E4054
:101C6000B5434560456896798E40B6B235434560C8
:101C7000C5684F000326BE40B543C560D5794E0008
:101C8000B540C6683543C560491C1029BFD3F0BDB7
:101C90004FF6FF7101600021017141718171C171C5
:101CA000704708B54FF480320092009A0A430092C0
:101CB000009AC261C161009AC261C2690092C269A0
:101CC000009208BD0246002013690B400BB10120B1
:101CD00000E0002070470146086980B27047024664
:101CE000002053690B400BB1012000E00020704739
:101CF0000146486980B2704701837047418370474D
:101D00000AB1018300E04183704741617047426935
:101D10004A4042617047F0B5002300244D07ED0EA4
:101D200002FA05F3CE1000F1200555F826504E07B3
:101D3000F70E0F26BE40B543CF1000F1200646F83F
:101D40002750CE1000F1200555F8265045EA03042F
:101D5000CE1000F1200545F82640F0BD00000240FD
:101D60000004024000080240000C02400010024043
:101D70000014024000180240001C024000200240F3
:101D800000240240002802400E49086070470D49B7
:101D9000486070470B49886070474AF6AA20094995
:101DA000086070474CF6CC40064908607047014611
:101DB0000020044AD2680A400AB1012000E0002055
:101DC0007047000000300040F948006840F0010012
:101DD000F74908600020F64908310860F4480068B7
:101DE000F4490840F2490860F348091D0860F348C7
:101DF000EF4984310860F0481038091D0860EC484C
:101E0000006820F48020EA4908600020E8490C318D
:101E10000860E7498C31086070470021E44A921C51
:101E2000117011460870704710B50146002200235A
:101E300000204A11012A02D1DD4C236808E0022A61
:101E400003D1DB4C7034236802E0D94C743423682E
:101E500001F01F02012494401C400CB1012000E05D
:101E6000002010BD38B5002000900024002500BFE0
:101E70003120FFF7D9FF05460098401C00900098DC
:101E8000B0F5A04F01D0002DF2D03120FFF7CCFFEC
:101E900008B1012400E00024204638BD014600209E
:101EA000C34A106820F0F80040EAC1001060704793
:101EB000C349086070470021BD4A7032117011702B
:101EC000012802D004280AD104E00121B84A703266
:101ED000117005E00521B64A7032117000E000BFB4
:101EE00000BF7047B7490860704770B5049C41EA6D
:101EF00082150126C6EB530645EA0645054345EA29
:101F00000465AB4E361D356070BDAD49086670473F
:101F1000820142EA0172A64B84331A607047A849D5
:101F20008866704710B5830143EA016343EA027390
:101F30009F4C8834236010BDA14908677047A049B1
:101F4000C864704702460020994B0833186820F097
:101F5000EC6042EA01031843954B08331860704760
:101F600002460020924B0833186820F0784042EA7D
:101F7000010318438E4B0833186070470146002058
:101F80008B4A0832106820F0030008431060704745
:101F900087480830006800F00C00704701460020B8
:101FA000834A0832106820F0F00008431060704740
:101FB000014600207E4A0832106820F4E0500843B1
:101FC0001060704701460020794A0832106820F4FA
:101FD000604040EAC10010607047F0B50021002267
:101FE0000024022500260223714F08373F6807F0BE
:101FF0000C0121B1042905D0082937D105E0724F21
:10200000076036E0714F076033E0694F3F1D3F685E
:10201000C7F38056664F3F1D3F6807F03F036EB120
:102020006A4FB7FBF3F7DFF888C10CF1040CDCF85A
:1020300000C0CCF3881C07FB0CF40CE0624FB7FB2C
:10204000F3F7DFF86CC10CF1040CDCF800C0CCF342
:10205000881C07FB0CF4564F3F1D3F68C7F3014730
:102060007F1C7D00B4FBF5F7076002E0564F076068
:1020700000BF00BF4E4F08373F6807F0F001090965
:10208000534F7A5C0768D7404760494F08373F682D
:1020900007F4E051890A4E4F7A5C4768D740876061
:1020A000434F08373F6807F46041490B484F7A5C5B
:1020B0004768D740C760F0BD002100F44072B2F518
:1020C000407F0AD13A4A0832116821F4F811414A96
:1020D00002401143364A08321160354A70321268A4
:1020E000C0F30B031A43324B70331A607047354903
:1020F00044390860704733494039086070473649B1
:102100000860704701460020294A8C32106820F090
:102110001F004A1E1043264A8C3210607047014649
:102120000020234A8C32106820F4F8504A1E40EAFE
:1021300002201F4A8C3210607047014600201C4A62
:102140008C32106820F4401008431060704701463C
:102150000020174A8C32106820F4400008431060B9
:10216000704701460020124A8C32106820F440303B
:1021700008431060704719490860704739B10C4A2C
:102180003032126802430A4B30331A6006E0084AC4
:10219000303212688243064B30331A607047F9B10F
:1021A000034A343212680243014B34331A601CE094
:1021B00000380240FFFFF6EA103000240030002013
:1021C00000004742800E47420024F40000127A00CB
:1021D00062000020FFFCFF0F5C014742E011474214
:1021E0008F4A126882438E4B1A60704739B18C4A0D
:1021F000121D126802438A4B1B1D1A6006E0884AB2
:10220000121D12688243864B1B1D1A60704739B13C
:10221000834A0C3212680243814B0C331A6006E089
:102220007F4A0C32126882437D4B0C331A60704730
:1022300039B17B4A103212680243794B10331A606D
:1022400006E0774A103212688243754B10331A60E9
:10225000704739B1724A243A12680243704B243BEA
:102260001A6006E06E4A243A126882436C4B243BA3
:102270001A60704739B16A4A203A12680243684BC3
:10228000203B1A6006E0664A203A12688243644B9B
:10229000203B1A60704739B1614A1C3A1268024308
:1022A0005F4B1C3B1A6006E05D4A1C3A1268824391
:1022B0005B4B1C3B1A60704739B1594A143A12689B
:1022C0000243574B143B1A6006E0554A143A126811
:1022D0008243534B143B1A60704739B1504A103A4D
:1022E000126802434E4B103B1A6006E04C4A103A0B
:1022F000126882434A4B103B1A60704739B1484A12
:102300001C3212680243464B1C331A6006E0444AF2
:102310001C3212688243424B1C331A60704739B139
:102320003F4A2032126802433D4B20331A6006E0D8
:102330003B4A203212688243394B20331A6070477F
:1023400039B1374A243212680243354B24331A60BC
:1023500006E0334A243212688243314B24331A6038
:10236000704739B12E4A2C32126802432C4B2C3361
:102370001A6006E02A4A2C3212688243284B2C331A
:102380001A60704739B1264A303212680243244B32
:1023900030331A6006E0224A303212688243204B02
:1023A00030331A607047012808D11D493C31096853
:1023B00041F008011A4A3C32116007E018493C31EB
:1023C000096821F00801164A3C321160704739B1A2
:1023D000134A273A12780243114B273B1A7006E042
:1023E0000F4A273A127882430D4B273B1A707047E9
:1023F0000B484030006840F0807009494031086067
:10240000704701460020064A283A12680A400AB17D
:10241000012000E00020704701492639087070470C
:102420003438024010B50446FB48844208D10121EB
:102430008014FFF752FF0021A014FFF74EFF3CE08D
:10244000F648844208D101210014FFF735FF00212E
:102450002014FFF731FF30E0F148844208D1012118
:10246000C013FFF729FF0021E013FFF725FF24E049
:10247000EC48844208D101214014FFF72EFF0021CF
:102480006014FFF72AFF18E0E748844209D10121D0
:102490000805FFF722FF00214FF48010FFF71DFF12
:1024A0000BE0E248844208D101214805FFF715FFFF
:1024B00000214FF40010FFF710FF10BD10B50022EF
:1024C000028802F441520B884C8823438C882343B2
:1024D000CC8823430C8923434C8923438C89234391
:1024E000CC8923431A430280838B4FF2FF7423402D
:1024F00083830B8A038210BD2DE9F04F0025022350
:1025000000244FF00109002200260027944690463F
:10251000B0F81CA04FF2400B0AEA0B0AA0F81CA06E
:102520004FF0020AA0F820A0858BD1F808A0BAF1DC
:10253000020F01D100BF82E0B1F804A0BAF1000F90
:1025400002D14FF0010901E04FF00209DFF8E0A2EB
:10255000DAF800A00AF4000ABAF1000F09D0DFF897
:10256000D0A2DAF800A02AF4000ADFF8C4B2CBF84F
:1025700000A0DFF8BCA20AF17C0ADAF800A0CAF3D6
:10258000881CDFF8ACA20AF17C0ADAF800A0CAF3D2
:102590000278DFF89CA2AAF1040ADAF800A00AF097
:1025A0003F07DFF88CA2AAF1040ADAF800A00AF4C7
:1025B000800ABAF5800F08D1DFF878A2BAFBF7FAE3
:1025C0000AFB0CFABAFBF8F607E0DFF86CA2BAFBDC
:1025D000F7FA0AFB0CFABAFBF8F6B1F806A0BAF55E
:1025E000007F0ED14FEA162A0AEB8A0A4FEA4A0AFE
:1025F000D1F808B0BAFBFBFA0AF1050A1FFA8AF211
:102600000FE04FEA491AB6FBFAFA0AEB8A0A4FEAD8
:102610004A0AD1F808B0BAFBFBFA0AF1050A1FFA18
:102620008AF24FF00A0AB2FBFAF202F00104A2EBBE
:10263000040ACAF34F034FF6FF7A0AEA0424022B76
:1026400001DBFF2B01DD02230024B1F806A04AEADA
:10265000040A4AEA030AA0F820A0B1F804A0B1F8DD
:102660000CB04AEA0B0AB1F802B04AEA0B0AB1F818
:1026700000B04AEA0B0A4AF4006A4AEA0505858373
:10268000BDE8F08F0021018041808180C1800181FF
:1026900041818181C1810721018270470021018030
:1026A00041808180C1800221816000218181704749
:1026B00021B1028842F04002028004E002884FF615
:1026C000BF731A400280704721B1828B42F480624E
:1026D000828304E0828B4FF6FF331A408283704777
:1026E00002884FF2FF731A40028002880A43028078
:1026F0007047B1F5804F04D1028842F480420280D5
:1027000004E002884BF6FF731A40028070474FF6D0
:10271000FF62914204D0028842F48072028004E099
:1027200002884FF6FF631A400280704721B1828809
:1027300042F00402828004E082884FF6FB731A4064
:102740008280704721B1828842F01002828004E0CA
:1027500082884FF6EF731A408280704730B50022AE
:102760000023848B4FF240052C4084830224048490
:10277000828B0C88B4F5007F01D00C8814B94FF41B
:10278000807308E00C88B4F5407F03D00C88B4F562
:10279000807F00D100238C888D892C434D882C4369
:1027A0001C4344F400642243828330BD014688897F
:1027B00070478181704721B1028842F40052028043
:1027C00004E002884DF6FF731A40028070470188CA
:1027D00041F480510180704702460020012901D058
:1027E000108B00E0908A70470146088A70471AB142
:1027F00083880B43838002E083888B438380704708
:1028000030B5002400230C110125A540ABB2AAB1BC
:1028100085881D43858014E0003001400038004069
:10282000003C004000340140005001400054014091
:102830000838024000127A000024F40085889D4385
:10284000858030BD0246002013890B400BB101206A
:1028500000E000207047CA4302817047F0B502468D
:10286000002000240023002501F00F070126BE40B0
:10287000B4B20B1101269E40B3B2968806EA030556
:102880001689264016B10DB1012000E00020F0BDF0
:1028900010B5002201F00F040123A3409AB2D343E4
:1028A000038110BD10B50446FE48844208D10121C1
:1028B0000846FFF712FD00210120FFF70EFD9DE005
:1028C000B4F1804F08D101210846FFF7F5FC002143
:1028D0000120FFF7F1FC91E0F348844208D1012187
:1028E0000220FFF7E9FC00210220FFF7E5FC85E06C
:1028F000EE48844208D101210420FFF7DDFC0021CD
:102900000420FFF7D9FC79E0E948844208D101218D
:102910000820FFF7D1FC00210820FFF7CDFC6DE077
:10292000E448844208D101211020FFF7C5FC0021B2
:102930001020FFF7C1FC61E0DF48844208D101218B
:102940002020FFF7B9FC00212020FFF7B5FC55E05F
:10295000DA48844208D101210220FFF7BEFC0021A1
:102960000220FFF7BAFC49E0D548844209D1012191
:102970000804FFF7B2FC00214FF48030FFF7ADFCF4
:102980003CE0D048844209D101214804FFF7A5FC6E
:1029900000214FF40030FFF7A0FC2FE0CA4884422A
:1029A00009D101218804FFF798FC00214FF4802011
:1029B000FFF793FC22E0C548844208D10121402062
:1029C000FFF77AFC00214020FFF776FC16E0C048B4
:1029D000844208D101218020FFF76EFC0021802075
:1029E000FFF76AFC0AE0BB48844207D10121801549
:1029F000FFF762FC0021A015FFF75EFC10BD00226E
:102A00000288A84B98420ED0AC4B98420BD0B0F144
:102A1000804F08D0A44B984205D0A44B984202D0D6
:102A2000A34B984204D14FF68F731A404B881A4338
:102A3000A04B984207D0A04B984204D04FF6FF43DA
:102A40001A400B891A4302804B68C3620B880385C6
:102A5000944B984202D0994B984201D18B7A0386CD
:102A60000123838270474FF0FF31416000210180D4
:102A700001814180817270470185828270470A46D8
:102A8000002101884FF68F73194011430180704770
:102A900041627047C16270470146486A704701460B
:102AA000088D704721B1028842F00202028004E0E2
:102AB00002884FF6FD731A400280704721B10288E8
:102AC00042F00402028004E002884FF6FB731A40D1
:102AD0000280704721B1028842F08002028004E047
:102AE00002884FF67F731A400280704702884FF6C3
:102AF000F7731A40028002880A43028070470288F6
:102B00004FF6FF431A40028002880A430280704752
:102B100021B1028842F00102028004E002884FF6EF
:102B2000FE731A400280704770B500240022002313
:102B3000058C4FF6FE7635400584028C8388048B25
:102B40004FF68F752C40B51E2C400D882C43751EFA
:102B50002A408D892A434D882A43524DA84202D0EB
:102B6000564DA84213D14FF6F7752A40CD892A4316
:102B70004FF6FB752A408D882A434FF6FF652B40A0
:102B80004FF6FF552B400D8A2B434D8A2B438380F4
:102B900004838D684563028470BD70B500240022F3
:102BA0000023058C4FF6EF7635400584028C838830
:102BB000048B48F6FF752C404FF6FF452C400D88DE
:102BC0004FF6FF7606EA05252C434FF6DF752A40BF
:102BD0008D8906EA05152A434D8806EA05152A431C
:102BE000304DA84202D0354DA8421DD14FF67F7519
:102BF0002A40CD894FF6FF7606EA05152A434FF69F
:102C0000BF752A408D8806EA05152A434FF6FF3521
:102C10002B404FF2FF752B400D8A06EA85052B43AA
:102C20004D8A06EA85052B43838004838D6885637E
:102C3000028470BD70B5002400220023058C4FF67D
:102C4000FF6635400584028C8388848B4FF68F7530
:102C50002C404FF6FC752C400D882C434FF6FF5549
:102C60002A408D894FF6FF7606EA05252A434D88CE
:102C700006EA05252A430B4DA84202D00F4DA84273
:102C800038D14FF2FF752A40CD894FF6FF7606EA1C
:102C900005252A434FF6FF352A408D8806EA05258B
:102CA0002A4319E0000001400004004000080040F1
:102CB000000C0040001000400014004000040140DF
:102CC000004001400044014000480140001800401D
:102CD000001C0040002000404EF6FF752B404DF6D2
:102CE000FF752B400D8A06EA05152B434D8A06EA2F
:102CF00005152B43838084838D68C563028470BD72
:102D000070B5002200230024058C4EF6FF76354076
:102D10000584038C8488828B48F6FF752A404FF621
:102D2000FF452A400D884FF6FF7606EA05252A431F
:102D30004DF6FF752B408D8906EA05352B434D88EE
:102D400006EA05352B43FE4DA84202D0FD4DA842B0
:102D500008D14BF6FF752C400D8A4FF6FF7606EA38
:102D600085152C43848082838D680564038470BD3F
:102D7000002101804180818081608181C181018247
:102D80004182704770B50346002000241846183071
:102D900001258D40ACB21D8CA5431D8409B10829C5
:102DA0000AD100EB610005684FF68F76354005606B
:102DB0000568154305600FE00D1FC5F34E05284457
:102DC000056848F6FF763540056005684FF6FF76E2
:102DD00006EA02263543056070BD41637047816392
:102DE0007047C1637047016470470A460021018B38
:102DF0004FF68F7319401143018370470A46002133
:102E0000018B48F6FF7319404FF6FF7303EA022364
:102E10001943018370470A460021818B4FF68F7357
:102E200019401143818370470A460021818B48F67F
:102E3000FF7319404FF6FF7303EA0223194381839E
:102E400070470A460021018B4FF6F7731940114372
:102E5000018370470A460021018B4FF2FF7319402E
:102E60004FF6FF7303EA02231943018370470A46B2
:102E70000021818B4FF6F77319401143818370470E
:102E80000A460021818B4FF2FF7319404FF6FF7302
:102E900003EA02231943818370470A460021018B0C
:102EA0004FF6FB7319401143018370470A46002116
:102EB000018B4FF6FF3319404FF6FF7303EA0223ED
:102EC0001943018370470A460021818B4FF6FB733B
:102ED00019401143818370470A460021818B4FF6C8
:102EE000FF3319404FF6FF7303EA0223194381832E
:102EF00070470A460021018B4FF67F73194011433A
:102F0000018370470A460021018BC1F30E014FF681
:102F1000FF7303EA02231943018370470A46002125
:102F2000818B4FF67F7319401143818370470A46A6
:102F30000021818BC1F30E014FF6FF7303EA0223D8
:102F40001943818370470A460021018C4FF6FD73B7
:102F500019401143018470470A460021018C4FF645
:102F6000F77319401143018470470A460021018C10
:102F70004FF6DF7319404FF6FF7303EA021319434C
:102F8000018470470A460021018C4FF67F73194077
:102F90004FF6FF7303EA02131943018470470A4690
:102FA0000021018C4FF6FF5319404FF6FF7303EADF
:102FB00002231943018470470A460021018C4FF215
:102FC000FF7319404FF6FF7303EA0223194301848C
:102FD00070470A460021018C4DF6FF7319404FF6E9
:102FE000FF7303EA023319430184704730B50023AD
:102FF00001248C40A3B2048C9C430484048C02FA08
:1030000001F5ADB22C43048430BD30B50023042457
:103010008C40A3B2048C9C430484048C02FA01F516
:10302000ADB22C43048430BD828B4FF2FF331A4083
:103030008283828B4FF6FF7303EA01231A43828354
:103040007047F0B50C461546002100220026078C7B
:103050004EF6FF7C07EA0C070784818B028C4FF643
:10306000FF7707EA043640F6FF4739404FF6FF770F
:1030700007EA052739434FF6FF7707EA0337394355
:1030800045F6FF773A4046F480573A4381830284FD
:10309000F0BD828B4FF6F3731A408283828B0A4312
:1030A00082837047F0B50C461546002100220026A9
:1030B000078C4FF6FF6C07EA0C070784818B028CA4
:1030C0004FF6FF7707EA04264FF60C7739404FF6A4
:1030D000FF7707EA03172F4339434FF2FF573A4070
:1030E00046F480773A4381830284F0BD028B4FF22D
:1030F000FF331A400283028B4FF6FF7303EA01236A
:103100001A4302837047F0B50C4615460021002291
:103110000026078C4FF6EF7C07EA0C070784018B2B
:10312000028C4FF6FF7707EA041640F6FF47394056
:103130004FF6FF7707EA033739434FF6FF7703E08F
:10314000000001400004014007EA052739434FF61B
:103150005F773A4046F010073A4301830284F0BD9E
:10316000028B4FF6F3731A400283028B0A430283E9
:103170007047F0B50C46154600210022068C4FF62C
:10318000FE773E400684018B028C4FF60C76314070
:103190007E1C06EA03162E4331434FF6F576324085
:1031A00044F00106324301830284F0BD70B5054648
:1031B0000C46208850B92389A28861882846FFF7E9
:1031C000D8FFE1882846FFF7CBFF25E020880428B8
:1031D0000AD12389A28861882846FFF794FFE188F5
:1031E0002846FFF783FF17E0208808280AD12389A3
:1031F000A28861882846FFF755FFE1882846FFF737
:1032000048FF09E02389A28861882846FFF719FF53
:10321000E1882846FFF708FF70BD0021018041804A
:10322000012181800021C180018170472DE9F04199
:1032300005460C4600260127608808B9022600E0F2
:103240000026A088012801D1022700E0012720885C
:10325000A0B92389A28861882846FFF78AFFE18800
:103260002846FFF77DFF23893A4631462846FFF777
:103270004AFFE1882846FFF739FF13E02389A28837
:1032800061882846FFF73FFFE1882846FFF72EFFB9
:1032900023893A4631462846FFF76BFFE1882846E6
:1032A000FFF75EFFBDE8F0810146486B70470146BD
:1032B000886B70470146C86B70470146086C7047C1
:1032C0000A884B881A438B881A43CB881A430B8988
:1032D0001A434B891A438B891A43A0F8442070473C
:1032E0000021018041808180C180018141818181F3
:1032F000704731B1B0F8442042F40042A0F84420B5
:1033000005E0B0F84420C2F30E02A0F84420704754
:1033100021B1828842F00402828004E082884FF664
:10332000FB731A408280704721B1828842F001020B
:10333000828004E082884FF6FE731A4082807047D4
:103340001AB183890B43838102E083898B43838194
:1033500070478182704702460020138A0B400BB1F0
:10336000012000E000207047CA430282704730B558
:103370000246002000230024158A05EA01039589EE
:1033800005EA010413B10CB1012000E0002030BDBA
:10339000CA430282704741EA0203A0F848307047EE
:1033A0001AB183890B43838102E083898B43838134
:1033B000704721B1828842F00802828004E082884E
:1033C0004FF6F7731A408280704701894FF6F87202
:1033D0001140018170470A46002101894FF68F7321
:1033E000194011430181704730B504460D46294606
:1033F0002046FFF7F0FF208940F00700208130BD14
:103400002DE9F04104460D4616461F46602D06D1B3
:103410003B46012231462046FFF775FE05E03B465C
:10342000012231462046FFF7A4FE29462046FFF739
:10343000D2FF208940F007002081BDE8F08130B53F
:103440000C4600210189C9B24FF6FF7505EA032534
:10345000154325432943018130BD2DE9F04105463F
:103460000E4617469846002443463A4631462846BB
:10347000FFF7E5FF2C894FF6F870044044F007048D
:103480004FF68F70044044F070042C81BDE8F08149
:10349000F0B504460D4616461F463B4632462946C1
:1034A0002046FFF7CCFF208940F480402081F0BD0A
:1034B00082884FF68F731A40828082880A43828006
:1034C000704702894FF6F8731A40028102890A4355
:1034D0000281704702894FF67F731A400281028988
:1034E0000A4302817047F0B50C4615461E4600217E
:1034F000002200230189028B038C4FF6F8773940B4
:1035000021434FF6FC473A4040F201173A434FF649
:10351000DD773B404FF6FF7707EA06172F433B4323
:10352000018102830384F0BD21B1828842F08002D0
:10353000828004E082884FF67F731A408280704751
:10354000A0F850107047000010B50446FA488442B5
:1035500008D101211020FEF7C0FE00211020FEF747
:10356000BCFE57E0F548844209D101214804FEF72A
:10357000A3FE00214FF40030FEF79EFE4AE0F04823
:10358000844209D101218804FEF796FE00214FF400
:103590008020FEF791FE3DE0EA48844209D10121F6
:1035A000C804FEF789FE00214FF40020FEF784FED8
:1035B00030E0E548844209D101210805FEF77CFE90
:1035C00000214FF48010FEF777FE23E0DF488442AD
:1035D00008D101212020FEF780FE00212020FEF7E7
:1035E0007CFE17E0DA48844209D101218807FEF702
:1035F00063FE00214FF08040FEF75EFE0AE0D548F2
:10360000844207D101214005FEF756FE00216005E6
:10361000FEF752FE10BD2DE9FF4705460E46002479
:10362000A14600BFA046B08900B100BF2C8A24F497
:103630004054F08804432C82AC8941F20C608443EE
:10364000B08831890843718908430443AC81AC8A4E
:1036500024F44074B0890443AC826846FEF7BDFC94
:10366000B548854202D0B948854202D1DDF80C90B8
:1036700001E0DDF80890A88900F4004040B109EBB2
:10368000C90000EB091031684900B0FBF1F707E011
:1036900009EBC90000EB091031688900B0FBF1F7B4
:1036A0006420B7FBF0F004012009642101FB1078CD
:1036B000A88900F4004040B1322000EBC800B0FB04
:1036C000F1F000F00700044308E0322000EB08109E
:1036D0006421B0FBF1F000F00F0004432C81BDE841
:1036E000FF874FF41651016000218180C180018164
:1036F0000C21418100218181704710B502460020D4
:10370000108A20F470600B884C8823438C882343F4
:10371000CC8823431843108210BD002101804180D2
:103720008180C180704721B1828942F40052828138
:1037300004E082894DF6FF731A4082817047028B44
:1037400002F47F420283028B0A430283704721B155
:10375000828942F40042828103E08289C2F30E0230
:103760008281704721B1828A42F40062828204E041
:10377000828A4FF2FF731A4082827047C1F30802B7
:103780008280704701468888C0F308007047028A2B
:103790004FF6F0731A400282028A0A43028270478F
:1037A00021B1828942F00202828104E082894FF6CF
:1037B000FD731A408281704782894FF2FF731A406D
:1037C000828182890A4382817047028A4FF6DF73C1
:1037D0001A400282028A0A430282704721B1028A99
:1037E00042F48042028204E0028A4BF6FF731A40E0
:1037F00002827047818941F001018181704721B1C6
:10380000828A42F00802828204E0828A4FF6F773CD
:103810001A4082827047028BD2B20283028B42EA44
:1038200001220283704721B1828A42F02002828203
:1038300004E0828A4FF6DF731A408282704721B11A
:10384000828A42F01002828204E0828A4FF6EF738D
:103850001A4082827047828A4FF6FB731A40828236
:10386000828A0A438282704721B1828A42F0020230
:10387000828204E0828A4FF6FD731A40828270478A
:103880001AB1838A0B43838202E0838A8B4383824B
:103890007047F0B50346002400260025002040F6BE
:1038A0006A17B94200D100BF1846C1F3421401F0B3
:1038B0001F06012707FA06F5012C01D10C3004E0A0
:1038C000022C01D1103000E014301AB107682F43E8
:1038D000076002E00768AF430760F0BD02460020C2
:1038E000B1F5007F00D100BF13880B400BB1012060
:1038F00000E00020704701F40072B2F5007F00D1B3
:1039000000BFCA430280704770B5024600240023FE
:103910000025002040F66A16B14200D100BFC1F375
:10392000421501F01F03012606FA03F3012D13D1FE
:103930009689334017E00000001001400044004029
:1039400000480040004C004000500040001401407E
:1039500000780040007C0040022D02D1168A3340DE
:1039600001E0968A33400C12012606FA04F4168808
:10397000344013B10CB1012000E0002070BD10B53F
:103980000022002340F66A14A14200D100BF0A12AF
:1039900001249440A3B2DC43048010BD00210160E7
:1039A000416070470146D1E90002904201D10120F7
:1039B00070470020FCE701464868401C41F288320D
:1039C00090FBF2F302FB13000A68904201D1012040
:1039D00070470020FCE770B504460E4615462046A9
:1039E000FFF7E9FF08B1002070BD04F1080162682B
:1039F00050182A46314600F0E3F86068284441F246
:103A0000883190FBF1F201FB120060600120EBE7CE
:103A100070B504460D4616462046FFF7C3FF08B1B1
:103A2000002070BD04F108002268111832462846B3
:103A300000F0C6F82068304441F2883190FBF1F282
:103A400001FB120020600120EBE770B50346002661
:103A500000251846FFF7A6FF08B1002070BD08E05A
:103A60001868401C18601846FFF79CFF08B100203A
:103A7000F4E703F108001968405CAA28F0D118683F
:103A8000401C03F108011860085C801C0E5C0224D5
:103A900006E003F10800005D2844C5B2601CC4B212
:103AA00003F108001968405C801CA042F1DCAE42C2
:103AB00001D00020D2E703F108001968405CC01C67
:103AC00003F10801085C552801D00020C6E71868FA
:103AD000401E18600120C1E770B5064600F0E0F80E
:103AE000056806F10B0020F00704B4429CBF0020DB
:103AF00070BD2B466A68BAB11068A04210D304F1B9
:103B0000080188423CBF5068586007D351681019BB
:103B100041601168091B016058601460101D70BD80
:103B200013465268002AE7D12146284600F0C0F823
:103B30000028DED170BD70B50446051F00F0B0F856
:103B40000068002C14BF446870BD002C18BFAC4244
:103B50003CBF20466468F8D301680A18AA4218BF1F
:103B6000456003D12A68054611440160286841195F
:103B7000A1421CBF6C6070BD616869602168084427
:103B8000286070BD0B4910B5A1F17C020A4CC2E956
:103B90003712372106E000EB104342F82130074B83
:103BA00000FB03400B1EA1F10101F4DC10BD01205C
:103BB000E8E70000943E0020E119D666CD0D010033
:103BC000032A40F2308010F0030C00F0158011F849
:103BD000013BBCF1020F624498BF11F801CB00F821
:103BE000013B38BF11F8013BA2F1040298BF00F875
:103BF00001CB38BF00F8013B11F0030300F0A280B5
:103C0000083AC0F0088051F8043B083A51F804CB58
:103C1000A0E80810F5E7121D5CBF51F8043B40F81E
:103C2000043BAFF30080D20724BF11F8013B11F829
:103C300001CB48BF11F8012B24BF00F8013B00F86D
:103C400001CB48BF00F8012B70474FF0000200B5D0
:103C5000134694469646203922BFA0E80C50A0E8AF
:103C60000C50B1F12001BFF4F7AF090728BFA0E85D
:103C70000C5048BF0CC05DF804EB890028BF40F829
:103C8000042B08BF704748BF20F8022B11F0804F6B
:103C900018BF00F8012B704770477047704700004D
:103CA00000487047043F00207047704770477047D6
:103CB00038B504460A4600206946AFF30080002864
:103CC00008BF38BD02460099204600F071F8012077
:103CD00038BD012000F086B8F8B5AFF30080054686
:103CE00000200C46102000BF0646A819A0420DD99E
:103CF000324669460020AFF30080070008BF00F09D
:103D000071F80098A04218BF0546C419FFF7C8FF14
:103D100005600746F01D20F007004619284600F010
:103D20000AF8B44208BFF8BDA21B31463868BDE8A6
:103D3000F84000F03DB800210160C0E90110704773
:103D40001020704710B5203AC0F00B80B1E8185031
:103D5000203AA0E81850B1E81850A0E81850BFF475
:103D6000F5AF5FEA027C24BFB1E81850A0E8185014
:103D700044BF18C918C0BDE810405FEA827C24BF68
:103D800051F8043B40F8043B08BF7047D20728BFF6
:103D900031F8023B48BF11F8012B28BF20F8023B45
:103DA00048BF00F8012B704700487047FC3E0020D8
:103DB000034640688C46002818BF88423CBF034633
:103DC0004068F8D318681844884207D00CF1030003
:103DD00020F00700001D411A521A0146081D0A6012
:103DE000FFF7A9BE10B500F039F8BDE8104000F0AB
:103DF0002FB870477546FFF7D7FFAE4605006946F6
:103E0000534620F00700854618B020B5FDF7F0FDB9
:103E1000BDE820404FF000064FF000074FF00008CB
:103E20004FF0000B21F00701AC46ACE8C009ACE84C
:103E3000C009ACE8C009ACE8C0098D46704710B5B0
:103E40000446AFF300802046BDE81040FCF7EBB914
:103E5000002801D000F02AB87047000010B50128F2
:103E600005D0002103A000F027F8012010BD09A112
:103E7000F8E7000053494752544D454D3A204F75DD
:103E800074206F662068656170206D656D6F727952
:103E9000000000003A2048656170206D656D6F720A
:103EA0007920636F7272757074656400014918201F
:103EB000ABBEFEE72600020070B505460C460A20A0
:103EC00000E06D1C00F011F835B128780028F8D119
:103ED00002E0641C00F009F814B120780028F8D141
:103EE000BDE870400A20AFF3008008B569468DF840
:103EF00000000320ABBE08BD4FF04070E1EE100A99
:103F000070470000243F00080000002074000000FB
:103F1000C4010008983F000874000020EC44000031
:103F2000E001000800000000007A030A0000000021
:103F30000000000001020304060708090000000059
:103F40001122334455050000450A0008810B000882
:103F50004F0B0008811100080098DC426111C0A8D5
:103F6000010AFFFFFF00C0A80101000002020202D7
:103F70000202020202020202020202020000000029
:103F80000000000000000000000001020304010224
:083F9000030406070809000004
:040000050800018965
:00000001FF
